:020000040800F2
:1000000000200020ED210008911E0008931E00082A
:1000100000000000000000000000000000000000E0
:10002000000000000000000000000000951E000815
:100030000000000000000000971E0008991E000844
:100040003D220008000000003D2200083D2200087B
:100050003D2200083D220008A51E0008AF1E000832
:1000600000000000B91E0008C91E00083D2200085B
:100070003D2200083D2200083D220008000000004B
:100080003D22000800000000000000003D220008A2
:10009000000000003D2200083D2200083D2200082B
:1000A0003D2200083D2200083D220008E11E000814
:0800B0003D22000800000000E1
:1000B80010B5064C2378002B07D1054B002B02D036
:1000C800044800E000BF0123237010BD5000002049
:1000D800000000005C620008044B10B5002B03D040
:1000E8000349044800E000BF10BDC04600000000FE
:1000F800540000205C6200080023C25C0133002A1F
:10010800FBD1581E7047000002B4714649084900E7
:10011800095C49008E4402BC7047C046002243086F
:100128008B4274D303098B425FD3030A8B4244D3B7
:10013800030B8B4228D3030C8B420DD3FF220902F9
:1001480012BA030C8B4202D31212090265D0030BB8
:100158008B4219D300E0090AC30B8B4201D3CB03AE
:10016800C01A5241830B8B4201D38B03C01A5241F0
:10017800430B8B4201D34B03C01A5241030B8B42F2
:1001880001D30B03C01A5241C30A8B4201D3CB02DD
:10019800C01A5241830A8B4201D38B02C01A5241C2
:1001A800430A8B4201D34B02C01A5241030A8B42C5
:1001B80001D30B02C01A5241CDD2C3098B4201D3DD
:1001C800CB01C01A524183098B4201D38B01C01A5B
:1001D800524143098B4201D34B01C01A52410309D2
:1001E8008B4201D30B01C01A5241C3088B4201D381
:1001F800CB00C01A524183088B4201D38B00C01A2E
:10020800524143088B4201D34B00C01A5241411A54
:1002180000D20146524110467047FFE701B5002061
:1002280000F0F0F802BDC0460029F7D076E7704725
:1002380003460B437FD4002243088B4274D303093F
:100248008B425FD3030A8B4244D3030B8B4228D3E0
:10025800030C8B420DD3FF22090212BA030C8B4206
:1002680002D31212090265D0030B8B4219D300E0A6
:10027800090AC30B8B4201D3CB03C01A5241830B2B
:100288008B4201D38B03C01A5241430B8B4201D3DB
:100298004B03C01A5241030B8B4201D30B03C01A04
:1002A8005241C30A8B4201D3CB02C01A5241830A7E
:1002B8008B4201D38B02C01A5241430A8B4201D3AD
:1002C8004B02C01A5241030A8B4201D30B02C01AD7
:1002D8005241CDD2C3098B4201D3CB01C01A52413E
:1002E80083098B4201D38B01C01A524143098B42C7
:1002F80001D34B01C01A524103098B4201D30B01B0
:10030800C01A5241C3088B4201D3CB00C01A5241D4
:1003180083088B4201D38B00C01A524143088B4299
:1003280001D34B00C01A5241411A00D20146524132
:10033800104670475DE0CA0F00D04942031000D351
:100348004042534000229C4603098B422DD3030AA6
:100358008B4212D3FC22890112BA030A8B420CD3B6
:10036800890192118B4208D3890192118B4204D3DF
:1003780089013AD0921100E08909C3098B4201D35F
:10038800CB01C01A524183098B4201D38B01C01A99
:10039800524143098B4201D34B01C01A5241030910
:1003A8008B4201D30B01C01A5241C3088B4201D3BF
:1003B800CB00C01A524183088B4201D38B00C01A6C
:1003C8005241D9D243088B4201D34B00C01A524143
:1003D800411A00D20146634652415B10104601D3D0
:1003E8004042002B00D54942704763465B1000D35A
:1003F800404201B5002000F005F802BD0029F8D000
:1004080016E770477047C0468446100062468C461F
:100418001900634600E0C0461FB500F065FF0028DC
:1004280001D40021C8421FBD10B500F0B5FE4042FE
:10043800013010BD10B500F057FF002801DB002087
:1004480010BD012010BDC04610B500F04DFF0028BA
:1004580001DD002010BD012010BDC04610B500F020
:10046800DDFE002801DC002010BD012010BDC046C3
:1004780010B500F0D3FE002801DA002010BD0120DD
:1004880010BDC0469E2110B5C905041C01F05CFAD8
:10049800002803D1201C00F0E1FA10BD9E21201C89
:1004A800C90500F02DF900F0D9FA80231B069C46F7
:1004B8006044F2E7F0B54F464646D646440245004A
:1004C800C0B5640A0F1C2D0EC60F002D00D18DE09B
:1004D800FF2D00D192E00023802099469A46E4003F
:1004E800C00404437F3D7802430A98467B001B0EF4
:1004F800FF0F002B00D170E0FF2B00D186E04246B1
:10050800D00080227F3BED180023D204024390469E
:100518009C4631004B467940681C0F2B1CD8764A04
:100528009B00D3589F4639004446E2465346022B67
:100538000FD0032B00D1D7E0012B37D100200024A6
:10054800C0052043C9070843E0BCBA46B146A846DF
:10055800F0BDFF200024F3E7260C2404220C4446B7
:100568002404240C434627001B0C574374435A4366
:100578005E4312193B0C9B189C4203D980225202FD
:10058800944666443F041A043F0CD2199401671E2E
:10059800BC411B0C920E9B1914439B011C431B016D
:1005A80000D49BE0012362081C40144302007F3200
:1005B800002A64DD630704D00F232340042B00D0F6
:1005C8000434230103D502004C4B80321C40FE2A20
:1005D800BFDCA401640AD0B2B2E74346002B3DD188
:1005E8004A4601331A4391469C4692E7002C29D18A
:1005F80004239946033B00259A4674E7002C1BD137
:1006080008239946063BFF259A466CE74346FF3583
:10061800002B0BD102234A461A4391469C4678E7A1
:1006280053463100022B00D083E792E703234A4662
:100638001A4391469C466CE70C239946093BFF25D3
:100648009A4650E7200001F089F97625431F9C401F
:1006580000236D4299469A462D1A44E7404601F018
:100668007DF94246431F9A4000232D1A90469C4626
:10067800763D4EE780240021FF20E40360E7012354
:100688009B1A1B2B00DD59E722009E30DA4084407C
:100698001300621E94411C43630704D00F232340B8
:1006A800042B00D0043463011AD50120002447E745
:1006B8008020C003044209D04346034206D1444681
:1006C800044364023900FF20640A39E78020C0032C
:1006D800044364023100FF20640A31E7280065E71B
:1006E800A4010020640A2BE78020C00304436402AD
:1006F800FF20640A24E7C04688620008FFFFFFF76E
:10070800F8B5CE46474643025B0A4E02DA009446E5
:10071800720A914645004A0080B52D0E1F00C40F8D
:10072800120EC90FB609FF2A5BD0012041408C4246
:1007380039D0A81A00285ADD002A6AD0FF2D00D126
:10074800D9E08022D20416431B2800DCE9E001200E
:100758006346181A430100D4B4E0800187093800C1
:1007680001F0FCF805388740854200DCCCE02D1A02
:10077800B5483840430704D00F230340042B00D06A
:100788000430430100D4A0E06A1CFE2D00D18DE0A6
:100798008001470AD2B2D0053843E4072043C0BCE1
:1007A800B946B046F8BDA81A8046002845DD002A9B
:1007B80070D0FF2D00D19EE08023DB041E4343460A
:1007C8001B2B00DCD2E00120604443017AD50135BF
:1007D800FF2D6BD001239D4A034040081040184369
:1007E800C8E7002E20D08C4223D02800FF380028EC
:1007F80039D0571B002D00D09DE06346002B00D157
:10080800DBE07B1E012F00D10DE1FF2F71D01F000F
:1008180098E0002E00D1A7E0421E012800D1E6E0B2
:10082800FF2868D010008FE701204140A14200D086
:100838007FE7FF2040428046A8444046002838D041
:10084800511B002D00D1AEE0FF2A00D1DFE080234C
:100858006046DB04184384461B2900DCD9E00120EC
:1008680015008019B1E7FE206A1C104271D1002DD5
:1008780000D0A6E06346002B00D1D9E00022002E6C
:1008880000D188E7981B430100D4E1E063460C00DF
:10089800F01A6FE7002E00D1B7E00200013A0128F4
:1008A80000D19CE0FF2826D0904688E7FF22002749
:1008B80071E7FE206A1C104264D0FF2AF6D01500AA
:1008C80066447008430700D056E7C308FF2D12D0CE
:1008D8005B025F0AEAB25EE76246002A00D196E050
:1008E800002E08D08022D203134204D0484610427A
:1008F80001D10C004B46002BD8D08027FF031F43A3
:100908007F02FF227F0A46E720233A00451B380072
:100918000135EA405D1BA840431E9841002510435D
:1009280028E720231B1A32009E40C2403000431E95
:10093800984110430CE7FF2ADBD080236046DB0494
:10094800184384461B2F56DD01200C001500301A71
:1009580000E763469F1B7B013DD4002F00D0FEE6D5
:1009680000240022002716E70500AFE732004346BF
:100978004146DA4020235B1A9E403000431E9841CE
:10098800104321E7002DA7D16346002B59D0002240
:10099800002E00D1FFE630006044430192D52A4B77
:1009A800013518408EE76346002B47D04B1E0129BE
:1009B80015D0FF292BD019004EE70C004B463D00FF
:1009C80084E76246002A8BD1002E92D1802700242A
:1009D800FF22FF03DFE663460C00F71ABFE630008C
:1009E80060440125430100D46CE70225F2E6634622
:1009F8000125981BAEE6202364466046FC40DF1BB9
:100A0800B840431E984120439FE705005EE74B46E8
:100A180071E7202365466046CD40591A8840431E39
:100A2800984128431CE763460C000125F01A91E61B
:100A3800002E95D00C004F460022ACE64B460D0028
:100A480044E74F460022A6E6FFFFFFFBFFFFFF7DBE
:100A5800002800D036E7002400279CE64102420027
:100A6800C30F490A0020120E7E2A03DD9D2A02DDEB
:100A7800094A98187047802000040143952A07DC2A
:100A88009620821AD1404842002BF3D10800F1E7A2
:100A9800963A9140F7E7C046FFFFFF7F70B5051E05
:100AA8000ED000F05BFF9E2304001B1A962B0CDC73
:100AB800082801DD083CA5406D026D0AD8B201E0A6
:100AC80000200025C005284370BD992B09DD0200D0
:100AD80029001B3291404A1E91410522121AD54025
:100AE8000D43052C12DC29000C4E31406A0709D051
:100AF8000F202840042805D004314A0102D59F233D
:100B080031401B1B89014D0AD8B2DBE7621F9540B3
:100B18002900024E31406A07F4D0E9E7FFFFFFFBE6
:100B2800F0B54F464646D6460D000400C0B51F0036
:100B380011002803620F400A10437A00520DE300A7
:100B48003C039146640AFA0F4F0F6E002743924602
:100B5800B846760DED0FC900954200D199E04C4694
:100B6800341BA446002C00DC7CE04A46002A00D155
:100B7800B8E0C54A964200D11CE180223C0012042C
:100B88001443A0466246382A00DD61E11F2A00DDD1
:100B9800CCE164462022121B444694400F00A14633
:100BA80064469140E7404C464A1E91413C434246C8
:100BB80021436446E240801A5C1AA3429B415F428B
:100BC800C71B3B0200D4D0E07F027F0A002F00D170
:100BD800FFE0380000F0C2FE01000839202322009F
:100BE8005B1A8F40DA408C401743B14200DAFFE0CD
:100BF800891B4B1C1F2B00DDA8E020223900D21ACC
:100C0800200094409140D840621E9441DF40002665
:100C180001430C43630709D00F232340042B05D05D
:100C2800231DA342A44164423F191C003B0200D487
:100C38009EE0954B01369E4200D1B7E0934AE40806
:100C480017407B0771057F0223433F0B4A0D1205AE
:100C58003A43ED072A4318001100E0BCBA46B146F2
:100C6800A846F0BD002C4BD04C46A41BA446002E31
:100C780000D023E104001C4300D1AFE16246541EBA
:100C8800012A00D115E2804DAC4500D1C8E1A44647
:100C98001BE14A46B21A9446002A00DCACE04A46F8
:100CA800002A43D0784A964200D1AFE180223C0026
:100CB80012041443A0466246382A67DC1F2A00DC67
:100CC8005FE14746203AD7406246202A05D064466D
:100CD8004022121B4446944021434A1E91410C0075
:100CE8003C4357E03A000A4300D105E12200013AAB
:100CF800012C00D182E1644CA4455BD0944641E7C5
:100D0800634C771C274200D0C4E004001C43002E2B
:100D180000D069E1002C00D1BFE144460C4300D06B
:100D2800D0E14207DB081343C00829E03A000A4330
:100D380000D170E162466446013A012C00D1E0E03E
:100D4800514CA44500D161E19446B4E73A001F39FB
:100D5800CA401100202B03D04022D31A9F403C43A5
:100D6800631E9C41002700260C43630700D053E70D
:100D7800B446E4087B072343F808434A94451DD04A
:100D88006246070352053F0B520D60E744460C4389
:100D9800621E9441E4189C429B415F423F183B020B
:100DA800E3D5394B01369E4200D0B5E0320000272A
:100DB80000234CE74207DB081343C0081A0002432C
:100DC80000D1E1E180273F0307433F032E4A3F0B51
:100DD8003DE7200000F0C2FD010018311F2900DCAA
:100DE800FCE60838844027000024B14200DBFFE617
:100DF800264A761A17400DE7002A2FD04A46921B3A
:100E08009446002E00D1ADE01F4A914500D10FE174
:100E18008022120410436246382A00DD0FE11F2A9F
:100E280000DD80E1644620221E00121B6746040094
:100E380093409440FE405A1E9341F84034431C436B
:100E4800804464188C42BF417F424E464744A6E71F
:100E580042460A4311004A1E9141ADE60C4C721CF1
:100E6800224200D0A1E002001A43002E00D0FAE08E
:100E7800002A00D145E13A000A4300D046E1420782
:100E8800DB081343C0087BE7FF070000FFFF7FFF75
:100E9800FE07000047465C1AC21BA342BF417F42BF
:100EA800B94617004A46BF1A3A0200D58DE023001A
:100EB8003B4300D08AE60020002561E7B44CA145F9
:100EC80000D1ADE08024240420436446382C3DDC66
:100ED80062461F2C00DDB7E020251E002D1B0400F4
:100EE800AB40AC40D640D04042465D1EAB41344397
:100EF800121A904623432CE04207DB081343C0082C
:100F08003BE75C189C429B4140445B42C718012662
:100F18003B0200D429E702269E4A630817400122B3
:100F280014401C43FB071C437F0873E64446203AE1
:100F3800D4406246202A05D067464022D21B474645
:100F4800974039434A1E9141214335E60343581ED1
:100F58008341CC1AA142BF4143467F4255464E4683
:100F6800DF1B2EE602001A4300D1BDE0624664464C
:100F7800013A012C00D1E5E0854CA44558D09446AF
:100F880049E764462022121B444694400F00A146BC
:100F980064469140E7404C464A1E91413C434246D4
:100FA8000C436146CA408018F4E6794CA24200D14D
:100FB800FDE6591899429B4140445F42C719FC0716
:100FC800490816000C437F08CFE6CC1AA142BF415E
:100FD80043467F42181A5546C71BF7E5C9087B07E1
:100FE80055460B43F808C8E6002C00D081E043467C
:100FF8000B4315D1802000250003E3E65C1AA342C9
:101008009B41C71B5B420126FF1ADAE54207DB0852
:101018001343C008D2E64207DB081343C008ACE616
:1010280043464246C9085B0755460B43D008C5E608
:10103800434642465B07C9080B43D008BEE6034354
:101048001C00631E9C41FCE60200203CE2401400A8
:101058006246202A03D04025AD1AA8400343581EF3
:101068008341234375E7002AE2D03A000A43CDD0F2
:101078004207DB0813438022C0081203104206D03F
:10108800FC08144203D12000CB087A0713435A0FF7
:10109800DB005207DB08134390E643460B4300D1BD
:1010A80009E743464246C9085B0755460B43D00843
:1010B80066E6CC1AA14289413F1A494255460126A3
:1010C8007F1A7EE542465C1A871AA3429241524231
:1010D800BF1A3A023DD5CC1AA1428941434649423A
:1010E8001F1A55467F1A95E57B07C9080B43F80870
:1010F80043E64446DB080C4330D142071343C0089B
:101108005CE67B07C9080B43F80839E65C189C4283
:101118009B4140445B42C7183B0200D425E61D4B67
:1011280001261F4021E60400203AD4406246202AC6
:1011380004D040226646921B904003435A1E9341B6
:101148001C437EE65C188C4289414044494247185A
:10115800DDE623003B4300D1ADE606E64407234322
:101168008024C0082403204208D04246D6082642DC
:1011780004D155463000CB0851070B435A0FDB000A
:10118800DB085207134319E60023014A1F005EE5F6
:10119800FF070000FFFF7FFFF0B54E464546DE46DD
:1011A80057469046E0B517001A03120B050084460F
:1011B80019480E034C0091465A00DB0F9B46360B2C
:1011C800640DC90F520D844219D0824210D00120FB
:1011D80094420ED14E450CD10120C44509D1594540
:1011E80017D0002C05D130002843431E984100E059
:1011F8000120F0BCBB46B246A946A046F0BD33006C
:1012080001202B43F5D1A242F3D14B463B43F0D109
:10121800E2E70020EDE7C046FF070000F0B54746CB
:10122800CE460400180016001B031B0B2D4D4A0068
:10123800994680B543000F03A446B0463F0B520DB4
:10124800C90F5B0DC00FAA4221D0AB4213D0002AB0
:1012580022D13C43002B02D14D462E4322D0002CF4
:1012680010D0814222D00220013908400138C0BC88
:10127800B946B046F0BD4D462E4329D1002AF0D1DB
:101288003C43EED10028F2D101204042EFE73D0077
:1012980025431DD19342EED0002BE2D14C46264384
:1012A800DFD1E0E70020002CE1D0DCE79A420ADC3D
:1012B800E8DB4F45D7D80ED000204F45D7D20029BC
:1012C800E2D00800D3E74342584140000138CEE756
:1012D80002204042CBE7C445C5D80020C445C6D249
:1012E800EDE7C046FF070000F0B54746CE460400CC
:1012F800180016001B031B0B2C4D4A00994680B59D
:1013080043000F03A446B0463F0B520DC90F5B0DB7
:10131800C00FAA420DD0AB4210D0002A27D13C43BF
:10132800002B11D14D462E430ED10020002C15D094
:101338000EE03D00254310D1934218D14D462E436F
:101348000BD1002A02D13C43002C0BD0814214D08F
:10135800022001390840013800E00220C0BCB9462B
:10136800B046F0BD0028F9D101204042F6E7002B35
:10137800ECD14C462643E9D1EAE79A4204DD4342E0
:10138800584140000138E9E79A42EBDB4F45DFD886
:1013980006D000204F45E1D20029E5D00800DDE75E
:1013A800C445D5D80020C445D8D2F5E7FF070000CA
:1013B800F0B557464E464546DE46E0B598460C031E
:1013C8004B000600924687B0240B5B0DCF0F002B15
:1013D80000D15CE1D94A934200D175E1420FE400A3
:1013E8001443802212041443D54AC500944663442A
:1013F8000093002399469B46434642461E03D20F5C
:101408005B0050469046360B5B0D00D120E1CB4A7D
:10141800934200D162E1CA49420F8C460099634465
:10142800F6008C46164380229C44120463461643F9
:10143800C200002000930099434601318C4649467A
:101448007B4001930F2926D8BE4B890059588F46F7
:10145800434601933400150083465B46022B16D0A1
:10146800032B00D103E2012B00D0CDE000220024A1
:101478000025019B12052243DB071A4328001100AF
:1014880007B0F0BCBB46B246A946A046F0BD002452
:101498000025AA4AEDE7280C2D042D0C2B00110C71
:1014A8001204120C5343984613002F0043439946E5
:1014B8004F434F44BB4647460B003F0CBA46434395
:1014C800DA440293D14504D980277F02B9464B44B8
:1014D800029353461B0C9B4653461F0443461B046A
:1014E8001B0C98463B0043440493330C3604360CDB
:1014F8009846330043439946434643432F009A4650
:10150800434677435D43380C4D444519A94503D9F3
:1015180080235B029946CA443F04280C3F0C2D04E3
:10152800ED19270C2404240C0300200050437A43AF
:1015380091463A0053440593030C9A464A43614343
:1015480049445144AB44894503D980235B029946F9
:101558004A4400040B0C000C0904091820009946A1
:10156800434670435C437E435F43030C9846A4198B
:1015780044444A440397A64204D980235B02984610
:10158800474403972304029E9A46059B5E44984667
:10159800AE42AD4176188E4289410004000C504499
:1015A80040446D424719B846934649428946C34468
:1015B800D94498428041A845AD4193459241894517
:1015C80089416D4240422843240C524249420A4311
:1015D800039B00198018C7184B46DC0D049B750245
:1015E8001D436A1E95414B46F60D7F0235435A024C
:1015F8003C431543FB0100D41CE101216A080D405E
:101608001543E207154364084F496144002900DC8B
:10161800B0E06B0709D00F222A40042A05D02A1D02
:10162800AA42AD416D4264191500E30104D5802139
:10163800464AC90014406144454A914200DD26E704
:101648006207ED08640249051543240B4A0D10E7AB
:101658005246324300D17FE0002E00D1DCE030005A
:1016680000F07CF902000B3A1D2301009B1A524638
:101678000839DA408E40164352468A40009B354965
:10168800181A03008C46634400200093D3E6250013
:1016980005434AD0002C00D1B0E0200000F05EF9EC
:1016A800010002000B391D2310005B1A31003500C0
:1016B80008388440D94085400C432648831A009353
:1016C800002399469B4697E60500254326D1082224
:1016D80000930223002491469B468DE65246009BC8
:1016E800324310D1154900268C466344494600937D
:1016F80002231943894602209DE65B460197022B87
:1017080000D0ADE6C3E60D4A0320944663444A463A
:10171800009303231A43914652468CE60C22009309
:101728000323050091469B4666E604239946002359
:101738000093013300249B465EE6C046FF07000085
:1017480001FCFFFFC8620008FF030000FFFFFFFE67
:10175800FE0700000DFCFFFF494601231943894697
:101768000026012067E6002380240025434A0193D0
:1017780024037EE60120401A382800DD76E61F287B
:101788005BDD1F2223005242511ACB40190020284A
:1017980003D03B4A6244944025436A1E95412A007F
:1017A8000A4307210D000024154011425BD00F2188
:1017B80000241140042953D0111D914292415242F4
:1017C800A4180A0023024BD501220024002550E664
:1017D80080231B031C4209D01E4207D133431C033C
:1017E80043461500240B254A019342E68022120342
:1017F80014432403214A240B01973AE600F0AEF87B
:1018080001000200153120321C2900DC4BE73400AE
:1018180008380025844050E700F0A0F803001A00BB
:10182800153220301C2A00DC1EE75646083B0022F1
:101838009E4023E7009B9C46E6E61249220061444D
:101848002E008D408A40C640691E8D4132432A438E
:10185800C4405307B6D00F2111400429ACD1B1E7D9
:1018680065076402240BD2081543002201E6802292
:10187800120314432403014A240BFAE5FF0700006E
:101888003E0400001E04000070B5002816D0C317DF
:10189800C5185D40C40F280000F060F8114A121AFC
:1018A8000A2816DC03002E0015339E400B23181A55
:1018B800C54052052D032D0B530D03E000240023D2
:1018C800002500261B052B43E4072343300019009D
:1018D80070BD0B38854052052D0300262D0B530D86
:1018E800F0E7C0461E040000844608006146FFE792
:1018F8001FB500F0BDF8002801D40021C8421FBD63
:1019080010B500F049F84042013010BD10B500F0A4
:10191800AFF8002801DB002010BD012010BDC04633
:1019280010B500F0A5F8002801DD002010BD012049
:1019380010BDC04610B500F055F8002801DC0020A5
:1019480010BD012010BDC04610B500F04BF80028AE
:1019580001DA002010BD012010BDC0461C21012362
:101968001B04984201D3000C10391B0A984201D37A
:10197800000A08391B09984201D30009043902A258
:10198800105C40187047C0460403020201010101BF
:10199800000000000000000070B5420045024E0241
:1019A8004C00C30F6D0A0120120E760A240EC90FCF
:1019B800FF2A06D0FF2C03D0A24201D1B54206D09F
:1019C80070BD002DFCD1FF2CFAD1002EF8D18B422E
:1019D80006D00120002AF3D12800431E9841EFE7E2
:1019E8000020EDE770B5420045024E024C00C30FDF
:1019F8006D0A120E760A240EC80FFF2A1BD0FF2C80
:101A08000ED0002A1BD1002C01D1002E1CD0002D95
:101A18000CD083421CD00221581E0840013870BDEA
:101A2800002E22D1002AF4D1002DF2D10028F6D1BF
:101A380001204042F3E7002D17D1FF2CF0D0002CF5
:101A4800E7D1002EE5D1E6E70020002DE7D0E2E758
:101A5800A24205DCEADBB54202D8E7D30020DEE784
:101A68004342584140000138D9E702204042D6E7B6
:101A780070B5420045024E024C00C30F6D0A120EAB
:101A8800760A240EC80FFF2A0BD0FF2C0DD0002A8F
:101A98001FD1002C16D1002E14D10020002D10D0FB
:101AA80009E0002D0CD1FF2C13D1002E08D1002AFB
:101AB80008D0834212D00221581E0840013800E0A5
:101AC800022070BD002DF4D10028FAD10120404237
:101AD800F7E7002CEDD1002EEBD1ECE7A24205DCB4
:101AE800F2DBB54202D8EFD30020EAE7434258417F
:101AF80040000138E5E7C0461FB50C22002101A8C7
:101B080004F09FFB8022184C184B12062261042215
:101B1800236080236261033A1B03A276E2612200FC
:101B2800636000232C3213700722626322002000B6
:101B38003C322383A360E3606362A3622363137070
:101B4800E36400F0CBFB002801D000F083F9084BD8
:101B580020000193012301A9029300F029FD002828
:101B680001D000F077F91FBD6C000020002401406F
:101B78000200000470B505008EB01422002103A8ED
:101B880004F05FFB1822002108A804F05AFB264B3A
:101B98002A689A4245D18023DB010893802308A84C
:101BA8001B060C9301F090FF002801D000F052F9B9
:101BB80080201E4B4003196C002601431964012143
:101BC8001A6C02400192019A5A6BA0200A435A6388
:101BD8005B6BC0050B400293029B022303935B18C7
:101BE80003A90493059601F09FFA114C114B2000AC
:101BF8002360052363607B33236180336361802323
:101C0800DB00A3612023E36180235B01A660E6601B
:101C1800236200F0E9FFB04201D000F01BF92C6507
:101C2800A5620EB070BDC0460024014000100240FD
:101C3800D00000200800024007B501200C4A916B33
:101C480001439163936B0221034000220193083002
:101C5800019B00F02FFF092000F056FF002202210F
:101C68000A2000F027FF0A2000F04EFF07BDC046FB
:101C780000100240F0B502270125A02689B01422E1
:101C8800002103A804F0DDFA394BF6055A6B300041
:101C98003A435A635A6B37493A400192019A5A6B50
:101CA80000242A435A635B6B2A002B400293029B51
:101CB80001F060FB30000022202101F05BFB2A00CC
:101CC80029002D4801F056FB0423300003A9039393
:101CD80004950594069401F027FA08230393C42376
:101CE80030009B0303A90493059401F01DFA2023F7
:101CF800300003A9039304950594069701F014FA9C
:101D08004023300003A903930494059401F00CFACE
:101D180080230393882330005B0303A9049305946D
:101D280001F002FA03A91448039504950594069452
:101D380001F0FAF9C0235B0103931123300003A9D2
:101D480004930594069701F0EFF922003900062064
:101D580000F0B0FE062000F0D7FE22003900072070
:101D680000F0A8FE072000F0CFFE09B0F0BDC04685
:101D78000010024004180000000400500848094BF5
:101D880010B5036003234360074BC360074B8360B0
:101D980001F012FB002801D000F05CF810BDC0462D
:101DA8002C01002000300040FF0F0000B80B00009D
:101DB80010B592B03422002105A804F042FA10228E
:101DC800002101A804F03DFA8020800001F02EFBDC
:101DD8000A230593F6330893002309930E930833D7
:101DE8000F9380239B0240221093802302240A929F
:101DF8009B053F3A05A80B920C940D94119301F0A2
:101E080041FB002801D072B6FEE707230390049037
:101E1800210001A80193029401F094FD002801D04B
:101E280072B6FEE712B010BD10B500F02DFAFFF73C
:101E3800BFFF04F0EBF8FFF71DFFFFF7FDFEFFF70C
:101E48005BFE00F0B9F800F0F3F8FFF797FF03F036
:101E580047FFFEE772B6FEE701200A4B82B0196C15
:101E68000143196480211A6C490502400092009AC6
:101E7800DA6B0A43DA63DB6B0B400193019B02B018
:101E88007047C04600100240FEE7FEE77047704703
:101E980010B500F00DFA04F0EBF810BD10B50820ED
:101EA80001F076FA10BD10B5802001F071FA10BD6E
:101EB80010B5024800F0FEFF10BDC046D00000205B
:101EC80010B5034800F0F6FF024800F0F3FF10BD1C
:101ED80088010020E401002070B5134C200002F0B6
:101EE8004FFB200002F08EFA102223680F4DD969AB
:101EF800114212D01A620E4A1378002B0DD10D4BE5
:101F08000D481B68596880235B425B1ADBB213706B
:101F180012782900D2B204F08BF92900802220001F
:101F280002F06CFF70BDC04640020020240500206E
:101F3800C5060020880100204506002070470000E3
:101F4800084B026882B09A4209D18020064A0002F2
:101F5800116C01431164136C03400193019B02B09F
:101F68007047C046002000400010024010B5040031
:101F780086B01422002101A804F063F90C4B2268F2
:101F88009A4213D101200B4A516B01435163536BA1
:101F980001A903400093009B1023A02001930E3B4E
:101FA8000293C0050233059301F0BEF806B010BDD8
:101FB800002000400010024010B588B01C2200210B
:101FC80001A804F03EF9174C174B184A2360022366
:101FD800636000232000A360E2602361A36101F035
:101FE800A3FF002801D0FFF735FF200001F0C6FF4E
:101FF800002801D0FFF72EFF60230193FA23002267
:102008009B00200001A902930392059202F01CF89C
:10201800002801D0FFF71EFF2000FFF7A7FF08B038
:1020280010BDC0463C01002000200040E70300002E
:1020380010B5184B184C0C22236096239B01636043
:1020480000232000A360E36023616261A361E36170
:1020580023626362A36202F047FE002801D0FFF703
:10206800F9FE0021200002F041FF002801D0FFF70F
:10207800F1FE0021200002F05DFF002801D0FFF7EB
:10208800E9FE200002F014FF002801D0FFF7E2FE6D
:1020980010BDC046003801404002002070B506005F
:1020A8008EB01422002103A804F0CBF818220021D6
:1020B80008A804F0C6F8334B32689A4260D101236D
:1020C80008A8089301F000FD002801D0FFF7C2FE20
:1020D80080202D4BC001196C0025014319641A6C2E
:1020E80002400192019A0222596B28481143596310
:1020F8005B6B03A913400293029BC02304920393D2
:1021080005950695079501F00FF8214C214B200005
:102118002360322363604E33236180235B01A56013
:10212800E5606561A561E561236200F05DFDA84297
:1021380001D0FFF78FFE331DDC67A662164B174CE4
:102148008022236033236360233BA3600023E36082
:102158006361A361E361802320005B012261236244
:1021680000F042FD002801D0FFF774FE1B2000227A
:102178000121F467A66200F09DFC1B2000F0C4FC5E
:102188000EB070BD0038014000100240000400503D
:10219800880100201C00024030000240E4010020B9
:1021A8000C4B026810B504009A4212D10A4A0B4936
:1021B800136C0B480B401364C02101F063F8231D16
:1021C800D86F00F06FFDE06F00F06CFD1B2000F091
:1021D800A7FC10BD0038014000100240FFBFFFFF00
:1021E800000400500D488546FFF7A8FE0C480D492D
:1021F8000D4A002302E0D458C4500433C4188C425A
:10220800F9D30A4A0A4C002301E013600432A242BF
:10221800FBD303F0E9FFFFF707FEFEE700200020ED
:102228000000002050000020B0630008500000208B
:1022380034070020FEE7000070B5104B0500197840
:10224800002901D1012070BDFA208000FDF766FF4A
:102258000B4B01001868FDF761FF00F071FC041ECC
:10226800F0D1032DEED8020001202900404200F0F1
:1022780021FC044B20001D60E5E7C0460400002057
:1022880000000020080000208023084A5B00116835
:1022980010B50B4303201360FFF7CEFF041E03D1D4
:1022A800FFF7DAFD200010BD0124FBE70020024003
:1022B800034A044B11681B785B1813607047C046CB
:1022C800D402002004000020014B18687047C04663
:1022D800D402002080684007C00F70470023F0B583
:1022E80085B0040001250393984200D1B7E0856DBD
:1022F8009D4205D1FFF73EFC23005433E5651D7070
:10230800802326685B05B2681A4200D1AAE0B36848
:102318000025DB0007D410230125A26D1343A36514
:10232800E36D2B43E3653000FFF7D4FF1022A36D64
:102338001340034300D0D0E0A36D6A4A1A40022339
:102348001343A36523689A68D20766D4227EA07EC9
:102358009203667E276B94464203A168F6030192B6
:10236800002F01D080277F01E268114362461143A4
:102378003143420311432269002A00DB87E05200FF
:10238800560822002C32127852000A43611CC97F79
:102398003A433243012905D1002800D07AE0802150
:1023A80049020A43616A002905D0E0204000014043
:1023B800A06A01430A43D9684B48E76C01400A43C5
:1023C800DA60220061683C3212788E0FB6079446B4
:1023D8003743012A09D1606C226C0243A06C3A434E
:1023E800024360463243104307001A693F480240DF
:1023F80080203A431A614A005208C00582420CD034
:1024080080221206914208D039483A4E026832407A
:10241800F026B603314011430160072070265A693F
:10242800616B82430A435A615869A26BB043120137
:1024380002435A612269002A34D1986A103A024349
:102448009A6207225B69134099423AD10023E365F7
:10245800A36D043A93431A0001231343A36528008C
:1024680005B0F0BDB26824490A401343B360234B5A
:1024780023491868FDF752FE013040000390039B82
:10248800002B00D143E7039B013B0393F7E780262A
:10249800B60376E72020A66D3043A065E06D0143C2
:1024A800E1657FE7802080038242CAD11C209A6AB6
:1024B800E269013A920002402C3890400200206EF6
:1024C800BDE71222A36D012593431A00102313437D
:1024D800A365E36D2B43E365C1E7A36D01251A43AB
:1024E800A265BCE7FDFEFFFF0102FEFF02FCFF1F25
:1024F80008270140FFFFC3FFE8FFFF6F000000202F
:10250800400D03007047704710B5806AFFF7FBFF66
:1025180010BD70474023806A10B5826D13438365F0
:102528000423C26D1343C365FFF7F3FF10BD00001A
:10253800502310B5846AA26D1A422CD1A26DB13312
:10254800FF331343A365C02320681B01C2681A42E6
:1025580014D1A37E002B11D103681B070ED5FFF7FA
:10256800B9FE00280ED10C21226853688B435360B2
:10257800A36D0E4A1A4001231343A3652000FFF7F9
:10258800C1FF10BD2023A26D1343A3650123E26D93
:102598001343E365F2E7A36DDB0603D52000FFF7DD
:1025A800B8FFEEE7236D5B6B9847EAE7FEFEFFFF97
:1025B8000023F0B587B00593030054331A7805005B
:1025C8000E000220012A00D1C3E001241C702868F3
:1025D800FFF780FE002800D0F9E004222F69736815
:1025E80097438022019312069446019A3368022A7F
:1025F80000D1C2E05903490B2A68029167450FD1FF
:10260800906A01439162B16854691802734E01409F
:102618003140844321435161002B64DB002095E065
:102628001F21019F0F40BC460F2761468F40F94389
:102638000391296EB9430F000299002914D1980E0D
:102648001F31084061468840019907438908E869B5
:1026580001312F668142D6D864469900090FA140FE
:10266800906A039C2040CCE72342EBD10221200052
:102678000B42E7D1080049180B42E3D10130190792
:10268800E0D40130D906DDD401309906DAD401301E
:102698005906D7D401301906D4D40130D905D1D47C
:1026A80001309905CED401305905CBD40130190534
:1026B800C8D40130D904C5D401309904C2D401303A
:1026C8005904BFD401301904BCD40130D903B9D49A
:1026D80001309903B6D480211800C90208400B4282
:1026E800B0D01220AEE7E0243D4A3E4811686404A9
:1026F8000C4083421AD180231B0419428ED11168E1
:102708003948014021431943384B1160186838494A
:10271800FDF704FD431C0C2058430590059B002B36
:1027280000D17BE7059B013B0593F7E731488342DE
:1027380011D18026080076043040314200D06DE780
:102748001168294B194021430E4316600023543564
:102758002B7007B0F0BD2848834200D05EE7802385
:102768000800DB031840194200D057E711681E4ED5
:10277800314021430B431360E8E7674505D12868DA
:102788005903826A490B8A438262002B00DB45E7C2
:10279800134A14481168834208D1A02310685B04C7
:1027A8001940114B03401943116037E71148834220
:1027B80003D1C02310681B04F2E70F48834200D0FE
:1027C8002CE7C0204004014013680748EAE72023AB
:1027D800AA6D20001343AB65B8E7C04600FFFF07AA
:1027E80008270140001000B0FFFF3FFE0000002056
:1027F800400D0300004000B8002000B470B504008C
:102808000068FFF767FD002801D1002070BD23682C
:102818009A68920705D49A680F49114010220A4312
:102828009A60FFF751FD0426050023689B68334230
:10283800EBD0FFF749FD401B0228F6D923689B68B7
:102848003342F2D010230120A26D1343A365E36D38
:102858000343E365DAE7C046E8FFFF7F0023F7B5E7
:1028680004000193036801209A68024201D0002005
:10287800FEBD9968224A114207D01023A26D134366
:10288800A365E36D0343E365F2E79A681D4D2A40AB
:10289800104398601C4B1B681B0223D4637E012BDA
:1028A800E5D0FFF711FD01260700226813683342BF
:1028B800DDD19368334203D193682B40334393604F
:1028C800FFF702FDC01B0228EFD923681B683342BB
:1028D800EBD11023A26D01201343A365E36D1E43C2
:1028E800E665C5E7094B0A491868FDF717FC01308A
:1028F8000190019B002BD1D0019B013B0193F8E78C
:1029080017000080E8FFFF7F082701400000002033
:10291800400D0300F8B5040000680D001600FFF72D
:10292800D9FC0223002840D1270054373A78012ADD
:102938003BD001223A702368D96811420CD19968BA
:10294800114205D09A681A49114002220A439A6036
:102958000122D9680A43DA602000FFF77FFF031ECF
:1029680023D1A26D13491140802252000A43A26567
:10297800E065114A206D2168C262104A0263104A5C
:1029880042631C220A603B704A68103313434B6051
:102998002A003300403100F0C9F9030020680449D7
:1029A8008268114004220A4382601800F8BDC046BC
:1029B800E8FFFF7FFEF0FFFF39250008112500081A
:1029C8001D250008036870B50400012099689A68FD
:1029D800024201D1002070BD02221142FAD1052124
:1029E8009D680D40012D1FD19968134801400A4385
:1029F8009A6003221A60FFF767FC060023689B6849
:102A08002B42E7D0FFF760FC801B0228F6D9236829
:102A18009B682B42F2D01023A26D01201343A365BB
:102A2800E36D1D43E565D6E71023A26D1343A36547
:102A3800E36D0343E365CEE7E8FFFF7F70B506006B
:102A48005436337805000224012B25D00123337036
:102A5800FFF7D4FE041E1DD1286D831DDB7F022BDA
:102A680007D100F0ADF9041E03D04023AA6D13432B
:102A7800AB6510212A68280053688B435360002CEB
:102A88000CD1FFF79FFF041E0BD001212A68D368E1
:102A98008B43D36000233370200070BDFFF792FF93
:102AA800F3E7AB6D024A1A4001231343AB65ECE729
:102AB800FEFEFFFF30B5FF2503242A000440E40092
:102AC800A24089012940D243A140C3B200280ADBB1
:102AD800C0240B4B80088000C018A40003591A407A
:102AE8001143015130BD0F200340083B05489B08A6
:102AF8009B001B18D86902401143D961F2E7C04610
:102B080000E100E000ED00E0002805DB1F2318408D
:102B18001E3B8340014A13607047C04600E100E055
:102B2800002809DB1F2318401E3B8340034AD36754
:102B3800BFF34F8FBFF36F8F7047C04604E100E0CB
:102B48008022431E5204012093420DD2C021074A1D
:102B580007485360036A09061B021B0A0B430362FA
:102B680000200723906013607047C04610E000E023
:102B780000ED00E0F0B5846CC56C6560046D002C58
:102B880002D0446D856D65601C25046C084E254097
:102B98000124AC4077683C437460046863608368D0
:102BA800102B02D1A260E160F0BDA160E260FBE7FA
:102BB8000000024010B50400036C094A9B089B18EA
:102BC8009B00436403681421D8B20838FDF7A6FABD
:102BD800044BA3641F2318401E3B8340E36410BDCD
:102BE800008200108008024070B504000120002C0B
:102BF80049D02568274B1421E818FDF78FFA0223DE
:102C08008000A61D2064F3772B68234AE1681340EF
:102C18002B60A3682A680B43216920000B43616974
:102C28000B43A1690B43E1690B43216A0B4313432F
:102C38002B60FFF7BFFF8023A268DB019A4201D116
:102C4800002363603F236268616C13400B60E06C93
:102C5800A16C013A4860032A16D8104A10489918FE
:102C68000322013B1340023A9A40A2651300002256
:102C78008900216560650A60436000200123E063E4
:102C88000534F377E07770BD002323656365A3659A
:102C9800F3E7C046F8FFFDBF0F80FFFF3F8200103B
:102CA80040090240F8B5012504002800002C34D062
:102CB800276814213B680026AB433B60174BF81884
:102CC800FDF72CFA1C238000206418402B00834059
:102CD800134A3E60516820000B435360FFF76AFFB8
:102CE800636CE26C1E60A36C5A6063685A1E032A08
:102CF80006D895400B495B189B001E600A4B5D6027
:102D08000020A31D20656065A065E0622063606304
:102D1800A063E0630534D877E077F8BDF8FFFDBF1E
:102D2800000002403F82001040090240F7B5451DEF
:102D38000193EE7F04000220012E34D00138E87799
:102D4800A71DFE7FB4466346F6B20096002683426E
:102D580031D10130F8772568E6632868009B9843ED
:102D68002860019B2000FFF705FF226B2368B24211
:102D78001AD00E2219680A431A60626C1168C903D6
:102D880004D580211068490001431160226D002A92
:102D980004D08021106849000143116001220020FD
:102DA80019680A431A60FEBD04211A688A431A602A
:102DB80019680A22DFE78023E363EE77F3E7000070
:102DC8000300F0B50120002B09D0981DC27F5C1DBF
:102DD800022A05D00422DA6300230120E377F0BD3C
:102DE8000E2519685E6C0A68AA430A603268114D9C
:102DF8002A40326001220E68944696430E601C21D8
:102E08001A6C0D4E114062468A4077683A437260E8
:102E1800D96C9A6C51601A6D002A05D01168294046
:102E280011605A6D9B6D53600123C3770020E077D2
:102E3800D5E7C046FFFEFFFF00000240F8B5811D40
:102E4800CB7F022B04D00423C363033B1800F8BDD7
:102E58000E240268154D1368076CA3431360012301
:102E680014689C431460446C22682A4022601C2425
:102E78003C40A3400E4A566833435360C26C836C8F
:102E88005A60036D002B05D01A682A401A60436DFA
:102E9800826D5A6001230024CB77431DDC77826B57
:102EA8001300A242D2D090472300CFE7FFFEFFFFD6
:102EB80000000240F8B51C210427046C264A214072
:102EC8003C008C40166803681D6826420FD03D42BE
:102ED8000DD01968890602D41968B9431960536876
:102EE8001C43036B5460002B1BD0984719E0022742
:102EF8003C008C40264215D03D4213D01968890603
:102F080006D40A251968A94319600121831DD977B8
:102F180053681C4354600022431DDA77C36A934206
:102F2800E3D1F8BD082427008F403E42F9D025425E
:102F3800F7D00E251C68AC431C6001231D008D4092
:102F48002900546821435160821DC363D37700224E
:102F5800431DDA77436BE2E7000002400630C07F8A
:102F6800C0B27047C06B70470020054B5A69824257
:102F780005DA044A9A60044A9A605869C00F704793
:102F88000020024023016745AB89EFCD8022044B26
:102F9800120659690A435A615869C043C00F7047FD
:102FA80000200240F8B504008027FFF78DF97F0262
:102FB8000619124D2B693B420BD12A69104B11009F
:102FC8001048194028611A4209D00F4B0120596056
:102FD80004E0FFF779F9B042EBD30320F8BDFFF71F
:102FE80073F980262418F6022B6918003040334202
:102FF800F4D0FFF769F98442F6D8EEE700200240E2
:10300800FA830000FB830000D8020020F7B5174EB2
:103018000193337804000D0002200092012B1ED08A
:103028000123FA203370002380007360FFF7BAFF92
:10303800002812D10E4F012C12D17B6923437B61EA
:10304800009B2B60BFF36F8F019B6B60FA208000A1
:10305800FFF7A8FF7B69A3437B6100233370FEBDA4
:103068002800009903F004F9F0E7C046D8020020D0
:1030780000200240044A05485369C9000340194327
:10308800034B1943516170470020024007E0FFFFDE
:1030980002000100F7B5214F05003B780224019199
:1030A800012B1AD00123FA203B70002380007B609B
:1030B800FFF778FF041E0ED104236B602B68042BE6
:1030C8000DD1FA20164A174B516980000B43536102
:1030D800FFF768FF040000233B702000FEBD0123BA
:1030E800019A5B421360AE68AB68EA689B18B3420A
:1030F8000CD968683100FFF7BDFFFA208000FFF7A0
:1031080051FF002808D00400019B1E600221044AD8
:1031180053698B435361DEE70136E5E7D8020020A7
:1031280000200240040001000023F0B585B00A68C1
:103138001400DC4001D105B0F0BD012514009D400C
:103148002C4001942A4200D18EE04A685E009446E1
:103158000322644622400324B440E4430294541EEC
:10316800012C2AD88768029C2740CC68B4403C438D
:10317800846044680127AC432500644624093C4028
:103188009C402C434460C568029C25408C68B44030
:103198002C43C460022A12D1DC080725A4000419B4
:1031A800276A03940F241D40AD00AC40A7430C6967
:1031B800AC402743039C276201E0032AE3D104685B
:1031C800029DB24025402C0014430460C02462468E
:1031D800A402224248D0254A03259C08A400A4182A
:1031E8000F221D40ED00AA40A027266EFF0596433A
:1031F8000022B8420CD01E4F0132B84208D01D4FF1
:103208000132B84204D01C4F0132B84200D0023219
:10321800AA40674632432266144C019A2668019DEB
:10322800D2433543FF0201D4350015406746256077
:103238006668019D3543BF0201D4350015406746D5
:1032480065600E4C019DE66F3543BF0301D4350020
:1032580015406746E5670A4C019EE56F2E43FF035C
:1032680001D415402E00E667013360E700180240DC
:103278000004005000080050000C005008180240DC
:1032880004180240F0B500230F0085B03A00DA4078
:1032980001D105B0F0BD01229A40140001923C40D2
:1032A800174253D02A4903259A08920052180F2131
:1032B8001D40ED00A940166E02910E400396A0260F
:1032C8000021F605B0420FD022498C460121604505
:1032D8000AD021498C460221604505D01F498C46F9
:1032E8000321604500D00231A940039DA94212D1B3
:1032F8001B4E1749F56FA543F5671A4EF56FA543A1
:10330800F5674D68A5434D600D68A5430D60116EC6
:10331800029CA1431166032459008C4007210F2603
:10332800194089008E400268019922430260DA0838
:1033380092008218156AB54315628268A2438260BA
:1033480042688A434260C268A243C26001339DE773
:10335800001802400004005000080050000C005003
:10336800041802400818024000690840431E9841AA
:10337800C0B27047002A01D0816170478162FCE7C2
:10338800426913000B401B04914319438161704744
:1033980070B5084D0400EB68184202D0E86002F0EE
:1033A80051F92B69234203D020002C6102F0EAF97D
:1033B80070BDC0460018024070B504000120002C02
:1033C80017D02368124A07251A60124A1A606268E1
:1033D8005A60A2689A60FEF777FF06002368DA68E9
:1033E800100028402A4205D11969E26891420CD0A0
:1033F8001A6170BDFEF768FF801B3128EED923687B
:10340800DB682B42EAD00320F3E7034A1A60F0E7AF
:10341800CCCC000055550000AAAA00000368024A57
:1034280000201A607047C046AAAA000010B5114CC7
:103438001149236802000B400343236080230020C6
:103448009B009A420ED10D4B0D491868062358432C
:10345800FCF764FE8022431CD2006169080010401A
:10346800114200D110BD002B01D0013BF5E703202C
:10347800F8E7C04600700040FFF9FFFF0000002099
:1034880040420F00F0B5040085B0002823D003683F
:10349800DB0710D423689B075ED423681B0700D57D
:1034A800C3E023685B0700D5F4E0E369002B00D094
:1034B8007AE1002029E03822AF4DAB681340EA6872
:1034C800102B0AD1D243930709D12B689B03E1D56E
:1034D8006368002BDED1012017E0082BF5D080228D
:1034E80063685202934212D12A6813432B60FEF795
:1034F800EBFE80270600BF022B683B42CAD1FEF7CD
:10350800E3FE801B6428F7D9032005B0F0BDA02195
:10351800C9028B4208D180232968DB020B432B6048
:103528002B681A432A60E2E72A6894490A402A600D
:103538002A6893490A402A60002BD8D1FEF7C4FEB6
:1035480080270600BF022B683B42A3D0FEF7BCFED3
:10355800801B6428F7D9D7E73823874DAA6813401A
:10356800EA68102B28D103210A40022A26D12A68AA
:10357800520502D5E268002AADD0696862698148BF
:10358800120201400A436A60002B0DD12B687E4A63
:103598001340226913432B602B687C4A9B045B0F02
:1035A800DA4013007A4A13607A4B1868FEF744FE33
:1035B800002800D171E78EE7002BD8D0E368002BF4
:1035C80020D02B68704A802713402269FF001343DC
:1035D8002B6080232A685B0013432B60FEF774FE80
:1035E80006002B683B4207D06A68636965491B027D
:1035F8000A4013436B6050E7FEF766FE801B022803
:10360800EFD981E72B68644A802713402B60FEF7C7
:103618005BFE0600FF002B683B4200D13DE7FEF74A
:1036280053FE801B0228F6D96EE73822524DAB684C
:103638001340182B08D12B6E9B0700D431E7A369E0
:10364800002B00D02DE746E7A2690123002A10D0FD
:103658002A6E022713432B66FEF736FE06002B6EF2
:103668003B4200D01DE7FEF72FFE801B0228F6D94B
:103678004AE72A6E02279A432A66FEF725FE0600C5
:103688002B6E3B4200D10CE7FEF71EFE801B022882
:10369800F6D939E73822384DAB681340202B08D1CA
:1036A800EB6D9B0700D400E7A368002B00D0FCE675
:1036B80011E780220021EB6B52050091134208D1DB
:1036C800EB6B1343EB63EB6B13400393039B0123F7
:1036D80000938027314E7F0033683B4215D0A368A2
:1036E800012B22D1EA6D1343EB65FEF7EDFD0227AE
:1036F8000600EB6D3B4238D0009B012B00D0D4E68E
:10370800EB6B274A1340EB63CFE633683B433360E8
:10371800FEF7DAFD019033683B42E0D1FEF7D4FDB5
:10372800019BC01A0228F6D9EEE6EA6D052B05D1F1
:10373800013B1343EB65EA6D0123D4E701218A437A
:10374800EA65EA6D03318A43EA65002BCDD1FEF7BD
:10375800BBFD02270600EB6D3B42CDD0FEF7B4FD62
:10376800104B801B9842F6D9CEE6FEF7ADFD0D4B07
:10377800801B9842BDD9C7E600100240FFFFFEFF3C
:10378800FFFFFBFFFF80FFFFFFC7FFFF0024F400E0
:103798000000002008000020FFFEFFFF007000402E
:1037A800FFFFFFEF8813000038213F4DAA680A4049
:1037B800102A53D03D4A022B38D12B68802713405A
:1037C8002B60FEF781FD0600BF042B683B4227D122
:1037D800616A236AEA680B43354980260A40134325
:1037E800E26AB6041343226B1343A26A120213431C
:1037F800EB6080232A685B0413432B608023EA680C
:103808005B051343EB60FEF75FFD04002B68334252
:1038180000D04EE6FEF758FD001B0228F6D973E6E5
:10382800FEF752FD801B0228CFD96DE62B68802653
:1038380013402B60FEF748FD0400B6042B681800FF
:103848003040334204D1EB681A4A1340EB605CE61F
:10385800FEF73AFD001B0228F0D955E6012B00D1EE
:1038680039E60322EB68216A1A408A4200D032E620
:103878007022616A1A408A4200D02CE6FE21A26AB0
:10388800C90119401202914200D024E6F822E16AE7
:1038980092031A408A4200D01DE6226B5B0F5B0739
:1038A800934200D105E616E600100240FFFFFFFE36
:1038B8008C80C11FFCFFFEEF382370B51E4CA26838
:1038C8001A4205D123681D489B045B0FD84070BD80
:1038D800A2681A40082A2AD0A2681A40102A1AD1C7
:1038E800E368E168DB434906490F7F2501319B07FF
:1038F8000CD1E36812481B0A1D40FCF70FFCE16875
:103908006843490F0131FCF709FCE0E7E3680B481D
:103918001B0A1D40F1E7A2681A40202A09D0A268B4
:1039280000201340182BD2D1FA20C001CFE7044859
:10393800CDE780200002CAE7001002400024F4000E
:1039480000127A00F7B504000D00002801D101200B
:10395800FEBD07274A4E33683B408B422AD3216875
:103968008B073BD4CB0748D4072733683B40AB428F
:103978000AD93368BB432B433360FEF7A5FC01909B
:1039880033683B40AB426BD123683E4D5B076FD435
:10399800FFF792FFAB683C4A1B051B0F9B009B5827
:1039A8001F221340D840394B1860394B1868FEF76E
:1039B80043FCCDE73368BB430B433360FEF784FC1D
:1039C800019033683B40AB42C9D0FEF77DFC019BB8
:1039D800C01A304B9842F4D90320B9E7294A4B075B
:1039E80004D5E0239068DB010343936093682A4879
:1039F8000340A06803439360B4E76268214F012A3B
:103A080019D13B689B03A2D50721BB688B4313439D
:103A1800BB60FEF759FC01903823BA681A40636806
:103A2800DB009A42A0D0FEF74FFC019BC01A194B4D
:103A38009842F1D9D0E7022A03D13B689B01E3D42D
:103A480085E7002A03D13B685B05DDD47FE70223C5
:103A5800032A03D1396E1942D6D178E7F96DFAE70E
:103A6800FEF732FC019BC01A0A4B984288D9B3E78B
:103A7800AB680A4A1340E2681343AB6088E7C04664
:103A880000200240001002400863000800000020E7
:103A98000800002088130000FFF0FFFFFF8FFFFFE2
:103AA800064B074A9B685B045B0F9B009B581F22D1
:103AB8001340044A1068D8407047C04600100240BE
:103AC8004863000800000020F0B505002B680020BE
:103AD80085B09B033BD58022484C5205E36B009090
:103AE800134208D1E36B1343E363E36B134003937F
:103AF800039B012300938027414E7F0033683B439B
:103B08003360FEF7E1FB019033683B4211D0E26D70
:103B1800C02311009B003B4E19401A4202D06B692A
:103B280099424DD1E36D00201E406B691E43E66546
:103B380006E0FEF7C9FB019BC01A0228E4D903205E
:103B4800009B012B03D1E36B2F4A1340E3632A68E0
:103B5800D30706D5032429494B6DA3436C68234337
:103B68004B65930606D52549284C4B6D2340AC6818
:103B780023434B6553040FD520492C694B6D9B009B
:103B88009B0823434B658023DB059C4204D180239B
:103B9800CC685B022343CB6013050FD5174A1C4C36
:103BA800536DE96823400B4353658023DB01994239
:103BB80004D18023D1685B020B43D36005B0F0BD0C
:103BC8008023E26DE06D11005B020343E365E36D62
:103BD800104831400340E365E165D307A2D5FEF7FD
:103BE80073FB07000222E36D13429BD1FEF76CFBC7
:103BF800094BC01B9842F5D9A1E7C0460010024006
:103C080000700040FFFCFFFFFFFFFFEFFFCFFFFF4B
:103C1800FF3FFFFFFFFFFEFF881300000122036A3A
:103C280070B593430362036A164A44688569154070
:103C38000A681543022293438A681343124A904242
:103C480005D0124EB04202D0114EB04213D1082610
:103C5800B343CE6833430426B343904205D00B4A9E
:103C6800904202D00A4A904205D10A4A8E692240FF
:103C78004C69344314434A68446085614263036273
:103C880070BDC0468CFFFEFF002C0140004401407F
:103C980000480140FFFCFFFF036A174A70B5134054
:103CA8000362036A154D4268C4692C400D682C43B1
:103CB800134D2B408D682D022B43124DA8420ED177
:103CC800114D1D40CB681B022B43104D2B40104D4E
:103CD8004E6915408A69324312012A4305E00D4DA9
:103CE800A842F4D00C4DA842F1D042604A68C461A1
:103CF800C263036270BDC046FFFEFFFF8CFFFEFF7C
:103D0800FFFDFFFF002C0140FFF7FFFFFFFBFFFF58
:103D1800FFCFFFFF0044014000480140036A124AF8
:103D280030B513400362026A104C4368C5692540E8
:103D38000C68240225430E4C22408C68240322433D
:103D48000C4CA04205D00C4CA04202D00B4CA04217
:103D580004D10B4C23404C69A401234343604B68B6
:103D6800C5610364026230BDFFEFFFFFFF8CFFFEF9
:103D7800FFDFFFFF002C01400044014000480140E4
:103D8800FFBFFFFF036A70B5104E114C334003624A
:103D9800026A4368456D25400C6825430D4C224056
:103DA8008C68240422430C4CA04205D00B4CA04242
:103DB80002D00B4CA04203D14C6933402402234368
:103DC80043604B6845658365026270BDFFFFFEFF77
:103DD8008FFFFEFFFFFFFDFF002C01400044014064
:103DE80000480140036A124A30B513400362026A70
:103DF800104C4368456D25400C68240225430E4C41
:103E080022408C68240522430C4CA04205D00C4C5F
:103E1800A04202D00B4CA04204D10B4C23404C6969
:103E2800A402234343604B684565C365026230BD05
:103E3800FFFFEFFFFF8FFFFEFFFFDFFF002C0140BA
:103E48000044014000480140FFFFFBFF020003005F
:103E580001203D321178814218D1022111701B686E
:103E6800DA680243DA600C4A934202D00B4A934262
:103E78000DD19A680A4900200A40062A06D0073957
:103E88008A4203D0012219680A431A6070471A68E7
:103E9800104318600020F9E7002C0140000400409E
:103EA8000700010070470000194A10B503689042E6
:103EB80002D0184CA04208D17024A3434C68234375
:103EC80090420BD0134CA04208D0134CA04205D00E
:103ED800124CA04202D0124CA04203D1114C2340F4
:103EE800CC6823438024A3434C69234303608B6835
:103EF800C3620B688362904205D0084B984202D097
:103F0800074B984201D10B6903630123436110BD3C
:103F1800002C014000040040002000400044014003
:103F280000480140FFFCFFFF70B504000120002C91
:103F380023D025003D352B78DAB2002B05D123009C
:103F48003C3320001A70FDF7FBFF02232B7020681A
:103F5800211DFFF7A9FF220001230020483213701A
:103F680047340A3A137053709370D37013715371B6
:103F78009371D371137223702B7070BD70B50400E8
:103F88000120002C23D025003D352B78DAB2002BF8
:103F980005D123003C3320001A70FFF783FF02236A
:103FA8002B702068211DFFF77FFF220001230020CE
:103FB8004832137047340A3A137053709370D370B1
:103FC800137153719371D371137223702B7070BD79
:103FD8001022036A70B593430362026A154C436862
:103FE800856925400C68240225432024A2438C6857
:103FF80024012243104CA0420FD18024A243140074
:10400800CA68120122434024A2430C4E4C691E4048
:104018008B6923439B00334305E0094CA042F4D04D
:10402800084CA042F1D043604B688561836302620B
:1040380070BDC046FF8CFFFE002C0140FFF3FFFF60
:104048000044014000480140F8B507003C373B7880
:1040580004000D0016000220012B0CD00138387026
:104068000C2A51D008D8042A2DD0082A3CD0002A7E
:1040780017D000233B70F8BD102A56D0142AF8D167
:104088002068FFF7AFFE802223681201596D0A43AA
:104098005A655A6D2D490A405A652A69596D1202A6
:1040A80051E02068FFF7BAFD0822236899690A439E
:1040B80004219A619A698A439A619A6929690A432B
:1040C8009A610020D5E72068FFF782FF80222368E5
:1040D800120199690A439A619A691C490A409A61CE
:1040E8002A6999691202EAE72068FFF7D5FD0421D9
:1040F8002368DA691643DE61DA698A43DA61DA69C4
:1041080029690A43DA61DCE72068FFF707FE8022A5
:1041180023681201D9690A43DA61DA690B490A404E
:10412800DA612A69D9691202EBE72068FFF72AFEEB
:1041380008222368596D0A4304215A655A6D8A4337
:104148005A655A6D29690A435A65BAE7FFFBFFFFAA
:104158001F2310B5012419408C408A40036AA343E9
:104168000362036A1A43026210BD000010B504001E
:10417800002906D1020001203E321378834249D03B
:1041880010BD0300042929D101203F331A78824247
:10419800F6D102221A702268D3680B43D3602068D4
:1041A8000122FFF7D5FF23682D498B4249D02D4ABC
:1041B800934246D02C4A934243D02C4A934248D14A
:1041C8009A682B4900200A40062AD9D007398A4222
:1041D800D6D0012219680A431A60D1E708290FD1FD
:1041E80040331B780120013B5A1E9341DBB2002B60
:1041F800C6D10223082913D1220040321370CAE71E
:104208000C2901D14133ECE7102901D14233E8E709
:104218004333E6E7022313702268D0680343BDE7FF
:104228000C2906D122004132137022681023D0686D
:10423800F4E7102903D1423401202370A0E7433466
:10424800FAE78022586C120202435A648B42B4D1B6
:10425800B6E70122196800200A431A6090E7C046B1
:10426800002C014000440140004801400004004087
:104278000700010010B5FFF779FF10BD30B5EFF367
:104288001084012282F31088C02501680B68AB43B3
:104298000B6084F31088EFF3108182F310880268B2
:1042A800044C93682340936081F31088202388305E
:1042B800036030BDFFFF7FFF30B5EFF310840122AC
:1042C80082F310880168134D0B682B400B6084F350
:1042D8001088EFF3108182F3108802680E4C9368FF
:1042E8002340936081F31088C36E012B0AD1EFF34A
:1042F800108183F31088102402681368A3431360A5
:1043080081F31088030020228C331A600023C366CF
:10431800436730BDDFFEFFFFFEFFFFEF70B505000E
:104328000120002D19D02E00242300248836336064
:104338002B681A6882431A6028001C605C609C60C5
:10434800FDF72EFF2B00200090331C60043B3460E7
:104358001C60EC662C6784352C7070BDF7B50500C1
:10436800883513002A6804000220202A32D1013837
:1043780000292FD0002B2DD08022A0685201904216
:1043880006D12269002A03D101321000114221D13D
:1043980022002600543221650027138053802122F1
:1043A800E06F903637602A60B84214D0226887637D
:1043B8000192114AC262114A0263114A4263019A88
:1043C8002832FEF7B3FCB84205D010230120336031
:1043D800DB182B60FEBD402223681A62EFF31081C0
:1043E800012383F3108822687F3390680343936026
:1043F80081F310880020EDE7B54400080745000860
:10440800174500080300020080218C32883370B5FC
:104418001B6815680268040092680A4220D0212BA4
:104428001ED1EFF31080203B83F310882268936835
:104438008B43936080F31088E06F00280DD0FEF75F
:10444800BFFC002809D0E06FFEF78CFD202804D1BE
:104458001023903423601D3870BD2000FFF70EFF35
:104468004021236800209B680B42F5D0222DF3D110
:10447800EFF31080012383F31088250004CD93689F
:104488008B43936080F31088E86F002808D0FEF70C
:1044980097FC002804D0E86FFEF764FD2028D7D0E9
:1044A8002000FFF709FF0020D6E7704703001B68CC
:1044B80070B51A6820231100806A19401A421AD16F
:1044C800030056331980EFF31084012282F3108819
:1044D800802501688B68AB438B6084F31088EFF309
:1044E800108182F310884023026810680343136028
:1044F80081F3108870BDFFF7D8FFFBE7704710B550
:10450800806AFFF7FBFF10BD70477047704770B5B2
:10451800846A2300220088338C321B68156822685D
:104528009268120608D5212B06D1230000225633A3
:1045380020001A80FFF7A2FE23689B685B0608D557
:10454800222D06D1230000225E3320001A80FFF7B7
:10455800B3FE220010239032116820000B43136031
:10456800FFF7D4FF70BD806A0023020010B55E32E9
:104578001380083A1380FFF7C9FF10BD7047000089
:10458800F7B50168C04DCB6904000A6888682B42FA
:1045980010D120252B4200D19AE0802676051540BF
:1045A8000640354300D193E0636F2000002B00D014
:1045B80083E083E0B54D0540AC466646B44D1540F2
:1045C800354300D184E001252B4207D0D60505D517
:1045D80026000D62903637683D4335602500022677
:1045E80090350195334207D0C50705D5019D0E6268
:1045F8002F68B6193E432E600426334209D0C507FA
:1046080007D527000E6290373E68350002262E43F4
:104618003E60082633420AD02027654617402F43BC
:1046280005D027000E6290373D682E433E608027F4
:1046380026003F0190363B4206D0550104D50F6253
:1046480020213768394331603168002936D020216C
:104658000B420AD01140802252051040014304D079
:10466800636F002B01D0200098472268019B4027E8
:104678001B68966828223E40134020001E4322D023
:10468800FFF71AFE23689B683B4218D0EFF31081AE
:10469800012383F31088250004CD9368BB439360FE
:1046A80081F31088E86F002809D07A4B8363FEF7FE
:1046B800C5FB002802D0E86F836B9847F7BD200040
:1046C800FFF724FFFAE7FFF721FF019B1E60F5E7DC
:1046D800E56E012D00D09EE01026334200D19AE00D
:1046E800324200D197E00E628B68402218001040D9
:1046F800134256D0201DC36F19684B689BB2002B1C
:10470800DCD027005C373F889F42D7D927005E3727
:104718003B80096820230F001F400197194232D1BE
:10472800EFF3108785F3108821685B4E09683140E4
:104738002668316087F31088EFF3108C85F31088B2
:104748002768B968A943B9608CF31088EFF3108C17
:1047580085F310882768B9689143B9608CF310888D
:1047680022008C321360019BE366EFF3108185F31E
:10477800108822680F351368AB43136081F31088E3
:10478800C06FFEF71DFB02232200236723005C3263
:104798005E331B881188C91A89B22000FFF7EEFE24
:1047A8008CE722005E32138812889BB2002A00D15F
:1047B80084E722005C321188C91A89B2002900D125
:1047C8007CE7EFF3108785F310882268334E13686F
:1047D8003340136087F31088EFF3108785F3108850
:1047E80022682F4E93683340936087F31088230024
:1047F80020228C331A60E0666067EFF3108085F33F
:104808001088102522681368AB43136080F3108862
:1048180002232367C1E780256D032B4206D0460299
:1048280004D520000D6200F03FFB47E780210B42D2
:1048380007D080252D0411402840084301D0A36FDC
:10484800B3E640210B4216D00A4214D0EFF3108091
:10485800012383F31088226813688B43136080F365
:1048680010882300202288331A6000232000A367C1
:10487800FFF71BFE22E7190214D5510012D52000BC
:1048880000F014FB1AE7C0460F08000001000010F2
:10489800200100046F450008FFFEFFFFDFFEFFFF59
:1048A800FEFFFFEFDB0100D408E7002A00DB05E785
:1048B800200000F0FAFA01E70123806A10B50367C7
:1048C800C36E012B06D103005C3319884908FFF732
:1048D80055FE10BDFFF719FEFBE7000003001B683B
:1048E80020221B6870B51900806A1140134234D128
:1048F80003005E331980EFF31085012383F31088DA
:1049080004681D4E21683140216085F31088EFF35B
:10491800108583F310880468A1689943A16085F322
:104928001088EFF3108483F31088402501688B68A2
:10493800AB438B6084F3108803008C331A60C36E1A
:10494800012B0AD1EFF3108183F310881024026839
:104958001368A343136081F3108800230367C36EB1
:10496800012B05D103005C331988FFF707FE70BDE2
:10497800FFF7CAFDFBE7C046FFFEFFFF70B5040066
:104988002569A168026829436569C36929431068D4
:10499800484D194328400143116051684648256A2B
:1049A8000140E06801435160A16990682943434D83
:1049B800284001430F209160D16A8143606A014316
:1049C800D1623F498A4215D103213E4A526D0A40BD
:1049D8008021013A0902022A5FD83B48805C8B4259
:1049E80014D0082857D8FBF78FFB0C56545651564D
:1049F80056563B0035498A424DD1802212029342D5
:104A08004DD0FFF74DF800284DD02BE0082842D8AC
:104A1800FBF77AFB45410841054141410900FEF792
:104A28004BFF3EE02A4B626A2A495200515A18004D
:104A3800FBF774FB656840006B08C0182900FBF79A
:104A48006DFB0200244B103A9A4224D80F2302002F
:104A580000079A4393B2400F22681843D06022E0BF
:104A680080200002636A1B4A5B00995AFBF756FBD9
:104A780065686B08C0182900FBF750FB0200164B4D
:104A8800103A9A4207D82368D8600CE0FEF714FF62
:104A9800B9E70F48E6E7012006E08B42B1D1FEF7FF
:104AA800FFFF031EBFD100200C4BA36600236367E2
:104AB800A36770BDF369FFCFFFCFFFFFFFF4FF11BE
:104AC80000380140001002406863000800440040BC
:104AD8000024F4006C630008EFFF000001000100EF
:104AE800836A30B5DA0706D50168284C4A6822403F
:104AF800C46A22434A609A0706D50168244C4A686A
:104B08002240046B22434A605A0706D50168214CAB
:104B18004A682240446B22434A601A0706D5016856
:104B28001D4C4A682240846B22434A60DA0606D547
:104B380001681A4C8A682240C46B22438A609A062C
:104B480006D50168164C8A682240046C22438A60A4
:104B58005A0610D50168134D4A68446C2A4022430E
:104B68004A6080225203944205D14A680E4C224082
:104B7800846C22434A601B0606D502680B495368B9
:104B88000B40C16C0B43536030BDC046FFFFFDFFB7
:104B9800FFFFFEFFFFFFFBFFFF7FFFFFFFEFFFFFB2
:104BA800FFDFFFFFFFFFEFFFFFFF9FFFFFFFF7FFA5
:104BB800F7B5802704000D00160001933F01226815
:104BC800D3692B405B1B59424B41B34201D00020B3
:104BD8002AE0089B0133F3D0FDF776FB019BC01A4E
:104BE800089B984201D8002B1FD1EFF310800122B7
:104BF80082F310882168204D0B682B400B6080F3EE
:104C08001088EFF3108082F3108821688B68934333
:104C18008B6080F310882200202388321360536051
:104C28000023032084342370FEBD042123681A68FE
:104C38000A42C4D0DA693A42C1D01F62EFF3108049
:104C4800012282F3108821680B4D0B682B400B6002
:104C580080F31088EFF3108082F3108821688B6846
:104C680093438B6080F310882200202388321360DE
:104C780053609360D4E7C0465FFEFFFF030073B53F
:104C88000026040090331E60FDF71EFB2368050014
:104C98001B681B0719D423681B685B070AD580218A
:104CA800104B0022009320002B00C903FFF780FF60
:104CB800002815D122000020202388321360536079
:104CC800E0662067843420700BE08021054B3200B9
:104CD8000093890303002000FFF76AFF0028DAD059
:104CE800032076BDFFFFFF0170B5041E01D101202E
:104CF80070BD050088352B68002B04D10200843272
:104D08001370FDF7CBF92423012122682B60136867
:104D180020008B431360FFF731FE0128E7D0A36A18
:104D2800002B02D02000FFF7DBFE236807495A68F2
:104D380020000A402A215A609A688A439A60012210
:104D480019680A431A60FFF799FFD1E7FFB7FFFF19
:104D5800F8B513000200060005005C3281650F00FB
:104D680013802221002290368C3532602960011D83
:104D78000400C86F904213D01D498263C1621D4967
:104D88003A0001631C49416321682431FDF7CEFFD5
:104D9800002805D0102301203360DB182B60F8BDF4
:104DA8002369002B0BD0EFF31081012383F31088C4
:104DB8002268FF3310680343136081F31088EFF310
:104DC8001080012383F3108821688A681A438A6057
:104DD80080F31088EFF3108183F3108822683F3343
:104DE80090680343936081F310880020D7E7C0469A
:104DF800E5480008C14800081745000803008C333F
:104E080070B51C680223202C25D1013B002922D033
:104E1800002A20D0802384685B019C4205D1036965
:104E2800002B02D10133194215D10023C366036850
:104E38005B681B020CD5EFF31085012383F3108800
:104E480080230468DB0426683343236085F31088D5
:104E5800FFF77EFF0300180070BD0000F8B5436E31
:104E68000400002B02D10D4B8366F8BD03680C4E7D
:104E78009F689B680B4D5B0FF05CE95CC000FBF71B
:104E8800D7F923006A3318803B015B0FF05CE95CBB
:104E9800C000FBF7CDF968342080E6E70100010087
:104EA8008C630008846300087047704770470000EF
:104EB80070B504008434227803000220012A11D03E
:104EC8001D002422012688352A601A681168106896
:104ED800B043106004480140002058662023116048
:104EE8002B60207070BDC046FFFFFFDFF8B50400DF
:104EF800250084352A7808000223012A18D00121C8
:104F080026002970226888362233336017681368B0
:104F18008B4313609368DB00D9080143916020003C
:104F2800FFF79CFF23681F602023336000232B704A
:104F38001800F8BDF8B5050084352B7804000A0080
:104F48000220012B18D02600242301382870883627
:104F5800336023681F681968814319609968074896
:104F68000140114320009960FFF778FF2368002073
:104F78001F60202333602870F8BDC046FFFFFFF193
:104F880000230270FA22437152000B1C914200D296
:104F9800131CC3807047F7B51F00490008AB1E7883
:104FA800CBB2141E0190009316D000F073FD009848
:104FB80000F032FE00F0B2FD451E200000F02CFE8D
:104FC80000F0ACFD6B425D41013843425841EDB2FF
:104FD8002D182C0000F080FD00F05CFD00980130D9
:104FE800C0B200F019FE00F099FD012801D101348A
:104FF800E4B2013EF6B2122E01D8002C05D000F022
:105008006BFD019B20001C71FEBD300000F036FED8
:1050180038700137EDE7F7B50C001E0008AB170034
:105028001D78019000F036FD6000C0B200F0F4FD7C
:1050380000F074FD0400380000F0EEFD00F06EFD95
:1050480001280FD1013C63425C41013400F044FD6A
:10505800019BE0B21871FEBD307800F0DDFD00F074
:105068005DFD0136012CF1D0013DEDB2122DF3D9D1
:105078000024EBE7F0B5030041180825FF2031268E
:105088008B4200D1F0BD1A7850402A0047B2440044
:10509800E0B2002F01DA7440E0B2013AD2B2002A3D
:1050A800F4D10133ECE7000037B5438804000A3334
:1050B8009BB243800A2B5CD94279002A0CD1012388
:1050C80043713233038103000232017808330092BE
:1050D800AA32FFF7A0FF37BD962B4AD9012A48D13B
:1050E8000223050043711C35053301780022009323
:1050F8002B00FFF750FF2379002B36D1062128001B
:10510800FFF7B8FFE31CDB7F8342E4D16722237FEC
:105118009343182BDFD1637FA07F1B02C018E57F64
:10512800000228180009FBF7B9FC1549FBF7C2F97A
:10513800D6218905FBF7BEF920630F20631C0540C3
:10514800D87F2D02A31C4019DD7F00022818FBF729
:10515800A5FC0C49FBF7AEF9D6218905FBF7AAF99E
:105168000949FBF7CDFA6063B5E70023236363635E
:10517800B1E7E2889A42AED2002363716380AAE75E
:105188000000C84200004843000048421022084B73
:1051980010B51B6819680A431A6050221A6200F099
:1051A80035FFFA2138220348C900FFF7E9FE10BD90
:1051B80040020020F4020020F7B5374C0121228874
:1051C80013004800205A98424DD8051C904200D937
:1051D800151CAAB20131FA29F3D1991A002904DD64
:1051E8002E4908881B189B1A0B802D4D2B785A1CAA
:1051F8002A70032B36D92B4B284F1C882A4B0521A4
:105208001E882A4B24B21B7836B25BB20193002366
:10521800F85EFBF70DF803B2254826495843FBF71B
:1052280007F80A216043FBF703F8019B86195E43E0
:10523800214B224A36B21E8010782149012814D108
:105248001B881BB20B8000233B802B700B881D48EA
:105258001BB2DA179B1853409BB21B4A83420CD9E6
:1052680096231380F7BD0300B4E71278002AEAD129
:105278001B88164A1BB21380E5E70B881BB2D917A7
:105288005B184B40FA219BB249008B4201D9642339
:10529800E7E72823E5E7C04630030020240600207E
:1052A8003F060020280600202606002017000020C0
:1052B800E40C0000FF0F00002A060020350600203D
:1052C8002E060020DC050000140000202C0600201B
:1052D800F0B50825012602000B4F0C4801390B4B8D
:1052E80089B2994200D1F0BD137858402B000400D0
:1052F8004008344001D0784080B2013BDBB2002B3B
:10530800F5D10132EAE7C04601A0FFFFFFFF000028
:10531800002130B58BB00C2207A8069100F091FF50
:10532800022301240293DB1803930B330493224BCB
:1053380006AD1A881B882A701B0A6B701F4B0594D0
:105348001A881B88AA701B0AEB701D4B1A881B88C9
:105358002A711BB21B126B711A4B1A881B88AA710F
:105368001BB21B12EB71184B1A881B882A721BB2CE
:105378001B126B72FDF7F8FD01A902A8FDF78AFE62
:10538800002802D0FDF702FE0AE02000069A079BDB
:105398000E49FDF73BFE002805D0FDF7F7FD032475
:1053A80020000BB030BD2000089A099B0849FDF782
:1053B8002DFE041EE6D0F0E72E0300204206002052
:1053C8002806002026060020320600200078000863
:1053D8000878000810B5012383F31088FFF798FFB9
:1053E800002383F3108810BD022330B5012487B051
:1053F800154D0293DB1803930A3304932B68059425
:1054080008332B60FDF7B0FD104B2A689A420AD981
:105418000F4B01A902A82B60FDF73CFE002802D023
:10542800FDF7B4FD0CE00B4B01201A882968002316
:1054380092B2FDF7EBFD041EF2D0FDF7A7FD0324A1
:10544800200007B030BDC04610000020D877000803
:10545800007000083C06002010B50400A0200122BE
:105468002021C005FDF786FF09490A48A2B2FEF7C8
:1054780075FF0948FDF772FD0128FAD1043000F0E4
:105488007BFEA02000222021C005FDF773FF10BD80
:10549800A405002040020020E4010020F0B55A4D88
:1054A8008BB0EB78A9781B026C790B432A795BBA2D
:1054B8009BB206212800240214430093FFF708FF3B
:1054C800030ADBB20193C3B20293504B64BA1A8841
:1054D8004F4BA4B25A804F4A127852B29A804E4A21
:1054E8001278DA804D4A12881A814D4A12885A81F8
:1054F8004C4A12889A814C4A1288DA814B4A12889F
:105508001A824B4A11784B4A090212780A435A8286
:10551800009AA2180A2A23DCAA7902998A421FD182
:10552800EA7901998A421BD143492A780A706A7834
:1055380003254A7062008A700022681CC0B2AE1C43
:105548000390F6B294422BD83B4FA9B23800FFF72C
:10555800BFFE039B7855000AF8543000FFF77CFF24
:10556800009BFF2B2DD1012C18D1274B02999A793A
:105578008A4213D1DB79019A93420FD1002405ADF9
:10558800142228002D4900F053FE2B4E2800FAF76C
:10559800B3FD844210D3C0B2FFF75EFF0BB0F0BD7D
:1055A800009810184000185E013207124F55039DED
:1055B800D2B248553500C0E72B5D33550134E4B20B
:1055C800E4E7009B0A2BE9D10F4B02999A798A42AA
:1055D800E4D1DA7901998A42E0D1174D1A7864004A
:1055E8002A705B78164A6B70138805211B0AEB70CA
:1055F80013882800AC702B71FFF76AFE6871000AE7
:10560800A8710720C8E7C046450600202A060020E2
:10561800C60600200C0000201600002042060020CC
:1056280028060020260600203C060020320600201E
:105638003606002044060020A405002094630008D4
:1056480030060020F8B50400A0204021C005FDF771
:105658008BFE3D4B80211870A020C005FDF784FE0D
:10566800802C38D1012831D1FCF72EFE374E0500A9
:105678003368C31A072B0FD8FA210420890000F0D9
:105688003DFD334F3B78012B06D1FA21022049001A
:1056980000F034FD00233B702B4B35601B78012B49
:1056A80003D12C4A1378013313702B4A1378013332
:1056B800DBB21370092B09D9264B28491878022820
:1056C80007D901200870002111701970244BDC6083
:1056D800F8BDFF20F6E7082CF8D10320214900F097
:1056E8000DFDA0202100C005FDF73EFE0128EDD1EB
:1056F8001D4B1E4A18701E4B1E491B8812880988AC
:105708001BB212B29B1A8B4210DD1B4A137801336D
:10571800DBB21370022BD9D9002118480170184840
:105728000170FA2BD2D903231370CFE7144A1378E8
:105738000133DBB21370022BC8D91049087000205E
:105748000D490870EDE7C0462C03002038060020FC
:105758001600002040060020340600201700002014
:105768000018024088130000350600202C0600208F
:105778002E06002014000020410600200C00002006
:105788003E060020010010B5082807D1A020C0055A
:10579800FDF7EAFD002801D1014B187010BDC04685
:1057A8003506002070B5204C05002000FEF7B6FD38
:1057B8001E4B2360012D2ED19623DB010C22636042
:1057C80000232000A360E36023616261A361E361B9
:1057D80023626362A362FFF787FA002801D0FCF70F
:1057E80039FB00212000FFF781FB002801D0FCF7DE
:1057F80031FB00212000FFF79DFB002801D0FCF7BA
:1058080029FB2000FFF754FB002801D0FCF722FBFE
:10581800FFF7BCFC70BD022D02D096239B01CDE79B
:10582800E1231B02CAE7C0464002002000380140BD
:10583800F7B5774CE378A1781B0265790B43227999
:105848005BBA9BB2062120002D0215430193FFF796
:105858003FFD06006F4F06222100380000F0E8FCEB
:10586800F3B2019A360AF6B26DBABB71FE710F2A0D
:1058780027D1A2799A4214D1E379B34211D1ABB2BC
:10588800013BF62B11D8644F3E883D80B6B2FFF736
:10589800A1FD002806D16378002B02D00820FFF76D
:1058A800DBFDF7BDF6B23E80FBE7FF2306213B7127
:1058B8007B712000FFF70CFDB871000A2378F8719E
:1058C800EAE7019A042A1BD1A2799A42E9D1E3793D
:1058D800B342E6D1FA23AAB29B009A42E1D84F4ECE
:1058E80034883580A4B2FFF775FD002855D10830FB
:1058F800FFF7B2FD4A4A338812689BB25363D0E778
:10590800019A28B2052A2BD1A2799A42C9D1E37902
:10591800B342C6D14349ABB25B18434A9BB29342E8
:10592800BFD8424C424B268819880A2309B25843EB
:10593800FAF77EFCABB200B2053B36B220800F2BE3
:1059480000D8258023881BB2042BAADD23881BB22C
:10595800142BA6DCFFF73EFD00289FD02680A0E789
:10596800019A062A1BD1A2799A4200D099E7E379D5
:10597800B34200D095E72B4AABB294462A4A634417
:105988009BB2934200D98CE72A4E3488358024B2E2
:10599800FFF720FD002800D180E7348081E7019AD5
:1059A800072A14D1A2799A4200D07AE7E379B34260
:1059B80000D076E7204B214A214C1A600022268825
:1059C800204B2580B6B21A80FFF70EFDC4E7019A76
:1059D800082A00D065E7A2799A4200D061E7E37906
:1059E800B34200D05DE7ABB2032B00D959E7164E9E
:1059F8003488358024B2FFF7EDFC0028CDD108307B
:105A0800FFF72AFD308800B2FFF7CCFE49E7C04611
:105A180045060020A40500202E0300204206002091
:105A28003C010020E40C0000C819000028060020F2
:105A38002A0600202606002010000020D87700083B
:105A48003C060020300600203206002010B50E4B20
:105A58000E491A7809888A420ED10D490978082911
:105A68000AD15B78032B04D0062B04D1FFF7E0FEA4
:105A780001E0FFF713FD10BD002AFCD1044A12789B
:105A8800082AF8D15B78EFE7450600202E030020AE
:105A9800C506002070B58026A0248025E40576017F
:105AA80031002D0120000122FDF764FC29000122AC
:105AB8002000FDF75FFC042000F076FB3100002297
:105AC8002000FDF757FC042000F06EFB290000229F
:105AD8002000FDF74FFC70BD70B58026A0248025FE
:105AE800E405360131006D0120000022FDF742FC7B
:105AF800290000222000FDF73DFC042000F054FBA3
:105B0800310020000122FDF735FC29000122200088
:105B1800FDF730FC042000F047FB70BD8021A02079
:105B280070B501224901C005FDF724FC012000F0F1
:105B38003BFB8021A02001220901C005FDF71AFCCA
:105B48008026012000F030FB65257601A020310079
:105B5800C005FDF709FC041E07D102008021A02022
:105B68000901C005FDF706FC06E0013DEDB2002D78
:105B7800ECD1FFF7B1FF0124200070BD70B580257E
:105B8800A0248026E4052D012900760120000022AA
:105B9800FDF7F0FB310000222000FDF7EBFB0220AF
:105BA80000F002FB290001222000FDF7E3FB0220A0
:105BB80000F0FAFA290020000022FDF7DBFB310093
:105BC80001222000FDF7D6FB70BD70B58025A0240A
:105BD8008026E4052D012900760120000022FDF72A
:105BE800C9FB310001222000FDF7C4FB042000F0AE
:105BF800DBFA290001222000FDF7BCFB042000F09D
:105C0800D3FA290020000022FDF7B4FB310001225D
:105C18002000FDF7AFFB70BDF8B580210400A0207F
:105C28000022A02680270901C005FDF7A3FB08254F
:105C3800F6053F0163B20122002B00DB0022802120
:105C480030004901FDF796FB022000F0ADFA012271
:105C580039003000FDF78EFB022000F0A5FA013D67
:105C6800002239003000FDF785FB64000220EDB208
:105C780000F09AFAE4B2002DDCD1F8BDF7B5802720
:105C8800A0260825002401903F01F60500223900CE
:105C98003000FDF76FFB022000F086FA3900300073
:105CA8000122FDF767FB8021640030004901E4B25E
:105CB800FDF75AFB002801D00134E4B2013D012070
:105CC800EDB200F071FA002DE0D1019B002B03D159
:105CD800FFF77BFF2000FEBDFFF750FFFAE700004B
:105CE800F7B5FFF753FAA54B1A88A54B1A801A88FF
:105CF800002A03D01988A34A914201D101221A80AF
:105D0800A14B1A88A14B1A801A88002A03D0198837
:105D18009C4A914202D1AF2292001A809C4C1B8867
:105D280022689BB253639B4B00229A5E9A4B1A805F
:105D38001A88002A03D01A8812B2013201D10A2225
:105D48001A80964B00229A5E954B1A801A88002A70
:105D580003D01A8812B2013201D100221A80914B65
:105D680000229A5E904B1A801A88002A03D01A885B
:105D780012B2013201D100221A80188800B2FFF74E
:105D880011FD8A4A8A4B7F4913608C460022894E4E
:105D98001F0019880837318035881989002D02D0ED
:105DA8003588654501D1002535804D1E8248ADB244
:105DB800854200D9002135888D4200D2C6E0002AEC
:105DC80001D07A4A13602000FEF740F80021200035
:105DD800FEF750FA794C2000FEF714FB80222000D1
:105DE8007749FFF70BF8774DFA2277492800FCF737
:105DF80091FDA02000222021C005FDF7BBFA322129
:105E0800002000F07BF9FA210120490000F076F922
:105E180003206E4900F072F9FA210420890000F08D
:105E28006DF90A21052000F069F90024002000F02E
:105E38008FF9002809D02800FCF700FEFFF7BCF90D
:105E4800FA2228006049FCF765FD012000F080F97E
:105E5800002809D000225E4B5E481A80FDF7DEFA62
:105E680001215D48FDF78CFA022000F071F9002845
:105E780033D0A0200421C005FDF782FAE1230134C4
:105E8800A4B25B019C4228D9338801339BB233808A
:105E980032883C4B9A4201D1002333804F4B1C7807
:105EA8004F4B1878FBF7F0FC009001911E2C59D845
:105EB8002000FBF7E9FC4B4A4B4BFBF779FA009AB9
:105EC800019BFAF7C1FA002804D0484A1388013325
:105ED8009BB21380FFF788FA0024032000F038F9FA
:105EE800002802D00222424B1A70042000F030F938
:105EF80000280BD0022000F017F9A020012204216D
:105F0800C005FDF737FA01223A4B1A70052000F058
:105F18001FF9002810D0384F3800FFF7C5F87B79F3
:105F2800022B09D1386BFAF7ADFA2D4B1870786B44
:105F3800FAF7A8FA294B1870304F3B78002B00D19C
:105F480074E7FFF783FD00233B706FE72C4B9F42FC
:105F580003D03B00012231801AE7002A00D132E742
:105F6800284B2EE76042FBF78FFC1E4A1E4BFBF7BF
:105F78001FFA0022244BFAF7D3FDA0E700780008A7
:105F88002E030020FFFF00000278000842060020D0
:105F98003C01002004780008280600200678000844
:105FA800260600200878000832060020100000208D
:105FB800007000083C060020FDFF000040020020A1
:105FC800240500206C000020300300208813000006
:105FD800DA0600202C0100200004005044060020AE
:105FE80036060020CDCCCCCCCCCC064030060020E8
:105FF8000C00002016000020F4020020C506002036
:10600800E0770008D877000800806640002370B564
:106018000C251C0012492800584301330A18546003
:10602800946054704454062BF5D1FA210D4B890025
:106038001868FAF773F8802301385B0498420DD288
:10604800C021094A090650600848036A1B021B0A56
:106058000B43036207239460136070BDFEE7C046DC
:10606800E40600200000002010E000E000ED00E061
:106078001C4A70B51368002B07D01368013B1360E6
:10608800002B02D10122184B1A7000220C25012680
:1060980016482C0054430319596800290AD0596836
:1060A80001395960002905D15E70215C012901D1AF
:1060B800996859600132062AEBD10D4B1A680132F2
:1060C8001A6019680B4A914201D100221A600A4AE3
:1060D80013780133DBB2092B01D8137070BD00238C
:1060E800FBE7C046300700202C070020E40600200C
:1060F800DC060020FFFFFF7FE0060020030030B52C
:10610800052800D9FEE7012585F310880C20002218
:106118005843044C2318596099605A70055582F306
:10612800108830BDE40600200300052800D9FEE7EA
:10613800012282F310880C2058430023034A1118C7
:106148004B604B70835483F310887047E40600203B
:1061580003000020052B09D80C305843054B0022BA
:106168001B185978C8B2012901D15A70704710001C
:10617800FCE7C046E406002000280FD0012800D123
:106188000130012383F310880022054B1860054B6A
:106198001A7082F310881A78012AFCD17047C04619
:1061A800300700202C0700200C4B70B50C49060066
:1061B8001868F9F7B3FF00230A4C46436568A168DD
:1061C800A2689142FCD05B18914205D99B1AB34250
:1061D80000D370BD1100F3E75B19F7E7000000205A
:1061E80040420F0010E000E070B500260C4D0D4C49
:1061F800641BA410A64209D1002600F02BF80A4D12
:106208000A4C641BA410A64205D170BDB300EB581C
:1062180098470136EEE7B300EB5898470136F2E7A6
:10622800A8630008A8630008A8630008AC63000816
:10623800002310B59A4200D110BDCC5CC454013380
:10624800F8E703008218934200D1704719700133B0
:10625800F9E70000F8B5C046F8BC08BC9E46704790
:10626800F8B5C046F8BC08BC9E4670470000000060
:1062780001B40248844601BC604700BF19000020F1
:106288006005000830050008300500082E050008E4
:1062980034050008340500087C0600082E050008AF
:1062A800340500087C060008340500082E0500089F
:1062B800280600082806000828060008B80600086E
:1062C8009E1400085C1400085C14000858140008A8
:1062D80062140008621400086E17000858140008B9
:1062E800621400086E1700086214000858140008A9
:1062F800021700080217000802170008D81700083C
:106308000000000000000000000000000000000085
:106318000000000000000000000000000000000075
:10632800010000000200000003000000040000005B
:106338000600000007000000080000000900000037
:106348000000000000000000000000000000000045
:10635800010000000200000003000000040000002B
:1063680004020800010002000400060008000A00F8
:106378000C00100020004000800000010804020406
:106388000801010101010103070100004443452DF3
:10639800323330322D56352E312E315F48414C0084
:0463A800E100000808
:0463AC00B90000082C
:1063B0000024F400010000000400000001000000BF
:1063C000007000084600010180220C4B30B55C696A
:1063D000D20222435A61EFF3108272B64C1CFF3492
:1063E000401A0D6845500431A142FAD1802149027A
:1063F00018690842FCD182F3108830BD00200240A9
:04000005080021EDE1
:00000001FF
